:020000040800F2
:1000000000060020E1010008F90E0008FD0E0008BE
:10001000550F0008FD0E0008290F0008E301000835
:10002000E3010008E3010008E3010008B928000823
:10003000E3010008E3010008E3010008E301000810
:10004000E3010008E3010008E3010008E301000800
:10005000E3010008E3010008453900087139000890
:100060009D390008C9390008F5390008E301000886
:10007000E3010008E3010008E3010008E3010008D0
:10008000E3010008E3010008E3010008E3010008C0
:10009000E3010008E3010008E3010008213A000839
:1000A000E3010008E3010008E3010008E3010008A0
:1000B000E3010008E3010008E3010008E301000890
:1000C000E3010008E3010008E3010008E301000880
:1000D000E3010008E3010008F51000080911000819
:1000E000893A0008E3010008E3010008E301000881
:1000F000E3010008E3010008E3010008E301000850
:10010000E3010008E301000855370008E301000897
:10011000E3010008E3010008E3010008E30100082F
:10012000E3010008E3010008E3010008E30100081F
:10013000E3010008E3010008E3010008E30100080F
:10014000E3010008E3010008E3010008A52F00080F
:10015000E3010008E3010008E3010008E3010008EF
:10016000E3010008E3010008E3010008E3010008DF
:10017000E3010008E3010008E3010008E3010008CF
:10018000E3010008E3010008E3010008E3010008BF
:10019000E3010008E3010008E3010008E3010008AF
:1001A000E3010008E3010008E3010008E30100089F
:1001B000E3010008E3010008E3010008E30100088F
:1001C000E3010008E3010008E3010008E30100087F
:1001D000E3010008E3010008E3010008E30100086F
:1001E00002E000F000F8FEE772B6394880F30888B4
:1001F000384880F3098838484EF60851CEF200019D
:10020000086040F20000CCF200004EF63471CEF2ED
:1002100000010860BFF34F8FBFF36F8F40F2000003
:10022000C0F2F0004EF68851CEF200010860BFF334
:100230004F8FBFF36F8F4FF00000E1EE100A4EF6C4
:100240003C71CEF200010860062080F31488BFF3F1
:100250006F8F02F06FFB03F005FA4FF055301F4926
:100260001B4A91423CBF41F8040BFAE71C49194A6A
:1002700091423CBF41F8040BFAE71A491A4A1B4B5A
:100280009A423EBF51F8040B42F8040BF8E70020F5
:100290001749184A91423CBF41F8040BFAE702F0B3
:1002A0004DFB03F049FA144C144DAC4203DA54F8F8
:1002B000041B8847F9E700F03FF8114C114DAC42A0
:1002C00003DA54F8041B8847F9E702F035BB000055
:1002D000000600200022002000000008000000208E
:1002E00000060020503F00080022002028220020A5
:1002F00028220020C4320020E0010008E0010008AC
:10030000E0010008E00100082DE9F04F2DED108A12
:10031000C1F80CD0C3689D46BDEC108ABDE8F08FD3
:10032000002383F311882846A047002001F040FFF6
:1003300001F060FE00DFFEE770B5204C0D230025C4
:1003400023706FF03F061F236570A570E57025715F
:100350006571A571E57125726672A372E57200F090
:10036000B3FC20B10F2325726672A372E57202F00E
:1003700075FA044602F09AFA0546D8B9104B9C4229
:100380001AD001339C4218BF054641F2883404BF9D
:1003900001250024002002F06BFA0DB100F05AF89C
:1003A00000F04AFD00F0BEFB204600F0B1F800F07E
:1003B00051F8F9E70024EDE70446EBE72822002096
:1003C000010007B008B500F02BFBA0F12003584254
:1003D000584108BD07B5054B02211B88ADF8043014
:1003E00001A800F089FB03B05DF804FB703B000836
:1003F00010B5202383F311881248C3680BB101F0B4
:100400005DFF0023104A0F484FF47A7101F01AFF84
:10041000002383F311880D4C236813B12368013B3B
:100420002360636813B16368013B6360084B1B780A
:1004300033B9636823B9022000F064FC322363609F
:1004400010BD00BF34220020F1030008502300201B
:100450004822002010B5254B254953F8042F0132BE
:1004600000D110BD8B42F8D1224C234B22689A4216
:100470003AD9224B9B6803F1006303F580439A420B
:1004800032D2002000F068FB1D4B0220187000F0F3
:100490002BFC1C4B1A6C00221A64196E1A66196E1A
:1004A000596C5A64596E5A665A6E5A6942F0800203
:1004B0005A615A6922F080025A615A691A6942F0F7
:1004C00000521A611A6922F000521A611B6972B651
:1004D0000D4A0E4B13601B682268202181F311889E
:1004E0009D4683F30888104710BD00BFFC3F0008FD
:1004F0001C40000804400008FF3F0008282200209C
:10050000482200200038024008ED00E000400008CA
:100510002DE9F04F99B0B34C01902022FF2110A893
:10052000A66800F02BFCB04A1378A346A3B9AF48E5
:100530000121C3601170202383F31188C3680BB1BC
:1005400001F0BCFE0023AA4AA8484FF47A7101F0DA
:1005500079FE002383F31188019B13B1A54B019A07
:100560001A60A54AA349019F0292002313704B60B1
:1005700099461C461D469846012000F0B5FB002F09
:1005800000F012829B4B1B68002B40F00D8219B0CB
:10059000BDE8F08F0220FFF715FF002840F0FB8137
:1005A000019BB9F1000F08BF1F46944B1B88ADF8A3
:1005B0002C3002210BA800F09FFADDE74FF47A708F
:1005C00000F02EFA031E0393EADB0220FFF7FAFE87
:1005D00082460028E4D0039B581E042800F2DD81E7
:1005E000DFE800F0030E1114170018A8052340F8E7
:1005F000343D042100F080FA54464FF0000856E0E4
:1006000004217848F6E704217D48F3E704217D487A
:10061000F0E71C24204600F0A1FA04340B900421DA
:100620000BA800F069FA2C2CF4D1E5E7002DB7D027
:10063000002CB5D00220FFF7C5FE0546002800F0CB
:10064000AF8101206C4C00F087FA0220207000F08E
:100650004BFB4FF000095FFA89FA504600F08CFA24
:10066000074658B1504600F097FA09F101090028F1
:10067000F1D12C46A9460027634B97E701230220BE
:10068000237000F023FB3E46DBF808309E4206D282
:10069000304600F063FA0130EBD10436F4E7029BF8
:1006A00000261E70534BA9465E602C46374600F06C
:1006B000B9FB15B1002C18BF0027FFF78BFE5BE7D5
:1006C000002D3FF46DAF002C3FF46AAF029B022077
:1006D000187000F009FB322000F0A2F9B0F1000A16
:1006E000C0F25E811AF0030540F05A81DBF8082061
:1006F00006EB0A03934200F25381BAF5807F00F2C1
:100700004F8155450DDA4FF47A7000F089F9049065
:10071000049B002BC0F244813C4A049BAB5401353E
:10072000EFE7C820FFF74EFE0546002800F03881AD
:100730001F2E11D8C6F12004544528BF544610ABD3
:1007400026F0030022463149184400F0EDFA224613
:10075000FF212E4800F012FB4FEAAA0A5FFA8AF244
:100760002A49304600F012FB0446002800F01A81A6
:1007700006EB8A0605469AE70220FFF723FE0028CB
:100780003FF40EAF00F02EFA00283FF409AF4FF00F
:10079000000A5346DBF8082092451CD2BAF11F0F1D
:1007A00012D8109A01320FD02AF0030218A90A4475
:1007B00052F8202C0B92184604220BA900F0DEFB05
:1007C0000AF1040A0346E5E75046039300F0C6F930
:1007D000039B0B90EFE718A8042140F84C3D00F074
:1007E0008BF964E7282200204C23002034220020CB
:1007F000F10300085023002048220020723B00082B
:100800002C22002030220020743B00084C220020C3
:1008100018A8002340F8343D642100F039F900287D
:100820007FF4BEAE0220FFF7CDFD00283FF4B8AE46
:100830000B9800F0C3F918AB43F8480D0421184693
:10084000CDE718A8002340F8343D642100F020F9DA
:1008500000287FF4A5AE0220FFF7B4FD00283FF486
:100860009FAE0B9800F0B8F918AB43F8440DE5E7DC
:100870000220FFF7A7FD00283FF492AE00F0C2F976
:1008800018AB43F8400DD9E70220FFF79BFD002885
:100890003FF486AE0BA9142000F0BAF9824618A8DE
:1008A000042140F83CAD00F027F951460BA896E72B
:1008B000322000F0B5F8B0F1000AFFF671AE1AF080
:1008C000030F7FF46DAEDBF808200AEB08039342B8
:1008D0003FF666AE0220FFF775FD00283FF460AEDC
:1008E0002AF0030AC244D0453FF4E1AE404600F08E
:1008F00035F904210A900AA800F0FEF808F104086E
:10090000F1E74FF47A70FFF75DFD00283FF448AE41
:1009100000F068F900283FF4AFAE109B01330CD013
:10092000082210A9002000F031FA00283FF4A4AEFC
:100930002022FF2110A800F021FAFFF74BFD3748D5
:1009400001F03CFC23E6002D3FF42AAE002C3FF4DE
:1009500027AE18A8002340F8343D642100F098F831
:10096000824600287FF41CAE0220FFF72BFD0028F2
:100970003FF416AE0390FFF72DFD41F2883001F0F1
:100980001DFC0B9800F098FA00F04CFA039B5746B8
:100990001C461D46F0E5054689E64FF00008FFE5D8
:1009A0002546FDE52C4667E6002000F039F8049066
:1009B000049B002BFFF6E3AD012000F087F9049BB8
:1009C000213B122B3FF6D8AD01A252F823F000BF15
:1009D00095050008BD0500082D06000879050008EA
:1009E0007905000879050008C1060008B10800086B
:1009F000790700081108000843080008710800087A
:100A0000790500088908000879050008030900082D
:100A1000AF0600087905000847090008A086010014
:100A20002DE9F34702AE00244FF47A7506F8014D24
:100A3000144FDFF85880454397F900305A1C5FFA8D
:100A400084F901D0A34212D158F82400036801228E
:100A5000D3F820A031462B46D047012807D10A4BB6
:100A60009DF8070083F8009002B0BDE8F0870134DC
:100A7000032CE1D14FF4FA7001F0A0FB4FF0FF30EE
:100A8000F2E700BF0022002098230020B43B0008BA
:100A90002DE9F0474FF47A75144FDFF85880064679
:100AA0004D43002497F900305A1C5FFA84F901D0B5
:100AB000A34210D158F8240003680422D3F820A0E0
:100AC00031462B46D047042805D1094B83F80090C6
:100AD0000020BDE8F0870134032CE3D14FF4FA7015
:100AE00001F06CFB4FF0FF30BDE8F08700220020E2
:100AF00098230020B43B000830B4074B1A78074B0A
:100B000053F822402368DD69054B0A46AC4601468E
:100B1000204630BC604700BF98230020B43B00084B
:100B2000A086010070B501F095FD094C094E2070BA
:100B3000002530682378834208D901F085FD3368A9
:100B400005440133B5F5804F3360F2D370BD00BF6B
:100B5000992300205823002001F032BE00F10060EC
:100B600000F580400068704700F10060920000F5D9
:100B7000804001F0BDBD0000054B1A68054B1B7895
:100B80009B1A834202D9104401F05EBD00207047D9
:100B9000582300209923002038B5074D04462868C3
:100BA000204401F059FD28B928682044BDE83840A8
:100BB00001F06ABD38BD00BF5823002010F00303C8
:100BC00008D1B0F5007F05D800F10050A0F508402D
:100BD0000068704700207047014BC058704700BF45
:100BE000107AFF1F064991F8243033B10023082200
:100BF000086A81F82430FFF7B7BF0120704700BFB3
:100C00005C230020014B1868704700BF002004E0FF
:100C100070B52A4B1C68C4F30B03240C63B140F27B
:100C20001342934231D040F2194293422FD040F206
:100C3000214293422DD10323214A0C2505FB032396
:100C40005D6893F9082042F201039C4224D0B4F578
:100C5000805F23D041F201039C4221D041F2030383
:100C60009C421FD041F207039C4208BF3122441E20
:100C70000C44013D0B46A3421ED215F9016F581CCE
:100C800096B1034600F8016CF5E70123D4E702238F
:100C9000D2E73F220B4DD6E73322E3E74122E1E7DB
:100CA0005A22E4E75922E2E72C2584421D7001D93B
:100CB000981C5A70401A70BD1846FBE7002004E0EB
:100CC000843B0008783B000800207047022802D1CE
:100CD000044B98617047012802BF024B4FF4006239
:100CE0009A61704700040240022804D14FF4003298
:100CF000034B9A6170470128FCD14FF00062F7E77F
:100D000000040240022805D1064A536983F0020319
:100D1000536170470128FCD1024A536983F4006390
:100D2000F6E700BF0004024010B50023934203D051
:100D3000CC5CC4540133F9E710BD000030B5441E4B
:100D400014F9010F0B4660B193F90050854201F18F
:100D5000010106D11AB993F90020801A30BD013A79
:100D6000EEE7002AF7D1104630BD000002460346E8
:100D7000981A13F9011B0029FAD17047024403465F
:100D8000934202D003F8011BFAE770472DE9F047C0
:100D9000234C94F8243005468846174683BB2E46DC
:100DA000DFF87C90C7B394F824302BB92022FF21C0
:100DB00048462662FFF7E2FF94F82400C0F10805D8
:100DC000BD4228BF3D465FFA85FAAD0041462A463E
:100DD00004EB8000FFF7A8FF94F82430A7EB0A0784
:100DE0009A445FFA8AFABAF1080F2E44A844FFB277
:100DF00084F824A0D6D1FFF7F5FE0028D2D108E070
:100E0000266A06EB8306B042CAD0FFF7EBFE002845
:100E1000C5D10020BDE8F0870120BDE8F08700BF04
:100E20005C230020024B1A78024B1A70704700BFF7
:100E3000982300200022002038B5184C184D204679
:100E400000F06CFC2946204600F094FC2D68154803
:100E5000EA6ED2F8043843F00203C2F8043801F015
:100E6000ADF91149284600F093FDEA6E0F48D2F81B
:100E700004380F4923F00203C2F80438A0424FF4AB
:100E8000E1330B6001D000F0A7FB0A48A04204D078
:100E90000749BDE8384000F09FBB38BDA82A0020B4
:100EA000C03C000840420F00E83C00081C24002021
:100EB000842300208426002038B50B4B1A780B4B76
:100EC00053F822400A4B9C4205460CD0094B0021A6
:100ED00018461422FFF752FF056001462046BDE880
:100EE000384000F079BB38BD98230020B43B00089F
:100EF000A82A002084230020FEE7000000B59BB054
:100F0000EFF3098168226846FFF70EFFEFF30583D0
:100F1000044B9A6BDA6A9A6A9A6A9A6A9A6A9A6A25
:100F20009B6AFEE700ED00E000B59BB0EFF309819E
:100F300068226846FFF7F8FEEFF30583044B9A6BCF
:100F40009A6A9A6A9A6A9A6A9A6A9B6AFEE700BFE4
:100F500000ED00E000B59BB0EFF309816822684620
:100F6000FFF7E2FEEFF30583034B5A6B9A6A9A6A26
:100F70009A6A9A6A9B6AFEE700ED00E030B5084D78
:100F80000A4491420BD011F8013B09245840013C1E
:100F9000F7D040F300032B4083EA5000F7E730BD61
:100FA0002083B8ED002304491A465A50C818083364
:100FB000802B4260F9D170479C230020026843686F
:100FC0001143016003B1184770470000024AD3681B
:100FD00043F0C003D360704700440040024AD36826
:100FE00043F0C003D3607047004800402DE9F04152
:100FF000D0F85C62F7683368DA0505469CB20DD517
:10100000202383F311884FF400710430FFF7D6FFDB
:101010006FF480733360002383F31188202383F3FC
:10102000118805F1040814F02F0333D183F31188DC
:10103000380615D5210613D5202383F3118805F131
:10104000380000F027FA002846DA0821281DFFF7AB
:10105000B5FF4FF67F733B40F360002383F31188A5
:101060007A060ED563060CD5202383F31188EA6C2B
:101070002B6D9A4202D12B6C002B2FD1002383F3CE
:101080001188D5F86422D368002B31D01069BDE8EF
:10109000F0411847230713D014F0080F0CBF0021AC
:1010A0008021E00748BF41F02001A20748BF41F07E
:1010B0004001630748BF41F480714046FFF77EFF5F
:1010C000A406736805D595F860122846194000F00B
:1010D00091FA3468A4B2A6E77060BEE727F0400733
:1010E0003F041021281D3F0CFFF768FFF760C5E79C
:1010F000BDE8F08108B50348FFF778FFBDE8084078
:1011000001F0EABB1C24002008B50348FFF76EFF7E
:10111000BDE8084001F0E0BB8426002010B5094C72
:10112000094A2046002100F035FA084BC4F85C3229
:10113000074C084A0021204600F02CFA064BC4F860
:101140005C3210BD1C240020CD0F0008004400407C
:1011500084260020DD0F00080048004038B5314DDE
:10116000037C002918BF0D46012B0446C0F86452C9
:1011700010D12D4B984242D12C4B1A6C42F40032C4
:101180001A641A6E42F400321A661B6E0B21262076
:1011900000F058F8264BD4F85C229A422B6802D013
:1011A00024498A423BD1244901EB5301B1FBF3F3BB
:1011B000A988080442BF23F0070003F0070343EAAD
:1011C00040039360EB8843F040039BB213612B898B
:1011D00043F001039BB2536141F4045343F02C03E9
:1011E000D36001F4A05100231360B1F5806F136840
:1011F00053680CBF7F23FF2384F8603238BD0F4B48
:101200009842C7D1094B1A6C42F480221A641A6EB4
:1012100042F480221A661B6E0B212720B8E708498A
:10122000C2E700BFE03B00081C2400200038024059
:10123000001001400014014000BD0105842600207B
:1012400080DE800200F1604300F01F02400903F5D8
:10125000614309018000C9B200F1604083F80013C6
:1012600000F5614001239340C0F88031036070476E
:10127000F8B5154682680669AA420B46816938BFEF
:101280008568761AB542044607D218462A46FFF703
:101290004BFDA3692B44A3610DE011D932461846DA
:1012A000FFF742FDAF1B3A46E1683044FFF73CFDD3
:1012B000E2683A44A261A3685B1BA3602846F8BDBC
:1012C00018462A46FFF730FDE368E4E783682DE916
:1012D000F041044693421546266938BF8568406947
:1012E000361AB5420F4606D22A46FFF71DFD63693E
:1012F0002B4463610DE012D93246A5EB0608FFF7D7
:1013000013FD4246B919E068FFF70EFDE26842445A
:101310006261A3685B1BA3602846BDE8F0812A4692
:10132000FFF702FDE368E4E710B50A440024C36157
:10133000029B006040608460C16081614161026124
:10134000036210BD08B582694369934201D1826886
:1013500082B98268013282605A1C42611970426906
:1013600003699A4201D3C3684361002100F042FF40
:10137000002008BD4FF0FF3008BD000070B52023ED
:1013800004460E4683F31188A568A5B1A368A26937
:10139000013BA360531CA36115782269934224BFCB
:1013A000E368A361E3690BB120469847002383F308
:1013B0001188284670BD3146204600F00BFF0028FA
:1013C000E2DA85F3118870BD2DE9F74F05460F4627
:1013D00090469A46D0F81C90202686F311884FF04C
:1013E000000B144664B1224639462846FFF740FFF9
:1013F000034668B95146284600F0ECFE0028F1D0BB
:10140000002383F31188A8EB040003B0BDE8F08F3C
:10141000B9F1000F03D001902846C847019B8BF318
:101420001188E41A1F4486F31188DBE7C1608161EB
:101430004161C3611144009B0060406082600161B2
:1014400003627047F8B504460E461746202383F31F
:101450001188A568A5B1A368013BA36063695A1C04
:1014600062611E70236962699A4224BFE368636106
:10147000E3690BB120469847002080F31188F8BD3E
:101480003946204600F0A6FE0028E2DA85F31188EE
:10149000F8BD0000836942699A4210B501D18268A3
:1014A0007AB98268013282605A1C82611C780369B1
:1014B0009A4201D3C3688361002100F09BFE20465D
:1014C00010BD4FF0FF3010BD2DE9F74F05460F4618
:1014D00090469A46D0F81C90202686F311884FF04B
:1014E000000B144664B1224639462846FFF7EEFE4B
:1014F000034668B95146284600F06CFE0028F1D03A
:10150000002383F31188A8EB040003B0BDE8F08F3B
:10151000B9F1000F03D001902846C847019B8BF317
:101520001188E41A1F4486F31188DBE702684368D8
:101530001143016003B11847704700001430FFF7F2
:1015400043BF00004FF0FF331430FFF73DBF0000F2
:101550003830FFF7B9BF00004FF0FF333830FFF7E6
:10156000B3BF00001430FFF709BF00004FF0FF3198
:101570001430FFF703BF00003830FFF763BF0000EF
:101580004FF0FF323830FFF75DBF0000002070479A
:10159000FFF7C4BD37B50F4B036000234360836082
:1015A000C360012304460374154600900B464FF4B4
:1015B000807200F15C011430FFF7B6FE00942B46F8
:1015C0004FF4807204F5AE7104F13800FFF72EFF7E
:1015D00003B030BDF43B000810B52023044683F36C
:1015E0001188FFF7BBFD02232374002383F31188C6
:1015F00010BD000038B5C36904460D461BB904216F
:101600000844FFF793FF294604F11400FFF79AFE00
:10161000002806DA201D4FF48061BDE83840FFF74E
:1016200085BF38BD026843681143016003B11847A4
:101630007047000013B5446BD4F894341A681178DD
:10164000042915D1217C022912D11979128901238B
:101650008B4013420CD101A904F14C0001F006FFAC
:10166000D4F89444019B21790246206800F0E0F907
:1016700002B010BD143001F089BE00004FF0FF33FE
:10168000143001F083BE00004C3001F05BBF00005D
:101690004FF0FF334C3001F055BF0000143001F023
:1016A00057BE00004FF0FF31143001F051BE000072
:1016B0004C3001F027BF00004FF0FF324C3001F0FA
:1016C00021BF0000D0F8942438B513681978042994
:1016D000054601D0012038BD017C0229FAD11279DA
:1016E0005C89012090400440F4D105F1140001F020
:1016F000E9FD02460028EDD0D5F894544FF48073EC
:101700002868697900F082F9204638BD406BFFF700
:10171000D9BF000000207047704700007FB5124B12
:101720000360002343608360C360012502260F4BE2
:10173000057404460290019300F184022946009644
:101740004FF48073143001F099FD094B019302941A
:1017500000964FF4807304F52372294604F14C007F
:1017600001F060FE04B070BD1C3C00080D170008BD
:10177000351600080B68202282F311880A7903EBE2
:10178000820210624A790D3243F822008A7912B13E
:1017900003EB8203186202230374C0F8941400233D
:1017A00083F311887047000038B5037F044613B1F6
:1017B00090F85430ABB9201D01250221FFF732FF0C
:1017C00004F1140025776FF0010100F01FFD84F88B
:1017D000545004F14C006FF00101BDE8384000F0B6
:1017E00015BD38BD10B5012104460430FFF71AFFBE
:1017F0000023237784F8543010BD000038B5044628
:101800000025143001F052FD04F14C00257701F061
:1018100021FE201D84F854500121FFF703FF2046CC
:10182000BDE83840FFF74EBF90F85C3003F060032E
:10183000202B19D190F85D20212A0AD0222A4FF0BE
:1018400000030ED0202A0FD1084A02650722426504
:1018500004E0064B036507234365002383650120ED
:10186000704703654365F9E70020704701220020B7
:10187000D0F8943437B51A681178042904461AD17F
:10188000017C022917D11979128901238B40134257
:1018900011D100F14C05284601F09CFE58B101A978
:1018A000284601F0E3FDD4F89444019B21790246D7
:1018B000206800F0BDF803B030BD000000EB8103EC
:1018C000F7B51C6A05460E46F4B1202383F3118850
:1018D00005EB8607201D0821FFF7A4FEFB685B6966
:1018E0001B684C3413B1204601F0CEFD01A92046FF
:1018F00001F0BCFD024648B1019B3146284600F08C
:1019000097F8002383F3118803B0F0BDFB685A6990
:101910001268002AF5D01B8A013B1340F1D105F172
:101920005C02EAE70D3138B550F82140DCB12023E4
:1019300083F31188D4F894241368527903EB82035B
:10194000DB689B695D6845B104216018FFF76AFE9A
:10195000294604F1140001F0BFFC2046FFF7B2FE57
:10196000002383F3118838BD7047000001F06CB884
:10197000012303700023436000F1240200F13801C9
:1019800042F8043B8A421361FAD1038143817047D4
:1019900038B50446202383F3118800254160C560D3
:1019A000056145618561C561056201F05DF802234D
:1019B000237085F3118838BD70B500EB81030546AF
:1019C0005069DA600E46144618B110220021FFF764
:1019D000D5F9A06918B110220021FFF7CFF93146DF
:1019E0002846BDE8704001F009B90000028902F004
:1019F00001020281428902F0010242810022026159
:101A000042618261C261026201F08CB9F0B400EB04
:101A100081044789E4680125A4698D403D434581DF
:101A200023600023A2606360F0BC01F0A7B900004E
:101A3000F0B400EB81040789E468012564698D40F6
:101A40003D43058123600023A2606360F0BC01F088
:101A500021BA000070B50223002504460370A0F8E7
:101A6000645080F8665080F8675005814581C560F4
:101A7000056145618561C561056280F84C5001F0E2
:101A800059F863681B6823B129462046BDE87040B9
:101A9000184770BD436802781B6880F868200522EB
:101AA00002700BB10421184770470000436890F89A
:101AB00068201B6802700BB10521184770470000B1
:101AC00090F84C3070B5044613B1002380F84C30C8
:101AD00004F15C02204601F047F963689B6863BB30
:101AE00094F85C5015F0600615D194F85D3005F05F
:101AF0007F0545EA032540F202339D4200F00E8146
:101B00005BD8022D00F0DC803FD8002D00F08780EC
:101B1000012D00F0CF800021204601F091FB002133
:101B2000204601F083FB63681B6813B10621204641
:101B30009847062384F84C3070BD2046984700280B
:101B4000CED094F8632094F8623043EA0223626DA9
:101B5000934238BF636594F95C30656D002B4FF09C
:101B6000200380F2FD80002D00F0EC80092284F833
:101B70004C2083F311880021636D226D2046FFF70E
:101B800057FF002383F3118870BDB5F5817F00F006
:101B9000B180B5F5407F49D0B5F5807FBBD194F8D1
:101BA0005E30012BB7D1B4F8643023F00203A4F8FF
:101BB000643026656665A665C3E740F201639D4211
:101BC0001ED8B5F5C06F3BD2B5F5A06FA3D1B4F860
:101BD0005C30B3F5A06F0ED194F85E3084F86630B7
:101BE000204600F0FFFF63681B6813B10121204607
:101BF000984703232370002323656365A365A0E74B
:101C0000B5F5106F32D040F602439D4252D0B5F583
:101C1000006F80D104F167032365012324E004F100
:101C20006403236502236365A5658AE794F85E3043
:101C3000012B7FF470AFB4F8643043F00203B6E7D1
:101C400094F86120616894F860304D6894F85F10F2
:101C500043EA0223204694F85E20A84700283FF478
:101C60005AAF4368236503686365A4E72378042BB0
:101C700010D1202383F311882046FFF7B7FE86F3A7
:101C80001188636884F867601B68032121700BB1B9
:101C90002046984794F85E30002BACD084F867302B
:101CA0000423237063681B68002BA4D00221204604
:101CB0009847A0E7374B23650223636500239DE720
:101CC00094F8601011F0800F204601F00F010ED043
:101CD00001F03CF8012806D002287FF41CAF2E4BFF
:101CE0002365606567E72D4B2365656563E701F054
:101CF0001FF8EFE794F85E30002B7FF40CAF94F8F8
:101D0000603013F00F013FF476AF1A06204602D57B
:101D100001F0AAFA6FE701F09DFA6CE794F85E30E3
:101D2000002B7FF4F8AE94F8603013F00F013FF40D
:101D300062AF1B06204602D501F082FA5BE701F094
:101D400075FA58E7142284F84C2083F311882B4647
:101D50002A4629462046FFF759FE85F3118870BDB3
:101D60005DB1152284F84C2083F311880021636D46
:101D7000226D2046FFF74AFE03E70B2284F84C2031
:101D800083F311882B462A4629462046FFF750FE4A
:101D9000E3E700BF4C3C0008443C0008483C000816
:101DA00038B590F84C300446152B29D8DFE803F0FD
:101DB0003E28282828283E28280B29392828282882
:101DC000282828283E3E90F8631090F86220436D42
:101DD00042EA01229A4214D9C268128AB3FBF2F590
:101DE00002FB15356DB9202383F311882B462A4653
:101DF0002946FFF71DFE85F311880A2384F84C302D
:101E000038BD142384F84C30202383F31188002339
:101E10001A4619462046FFF7F9FD002383F311887F
:101E200038BD836D03B198470023E7E7002101F037
:101E300007FA0021204601F0F9F963681B6813B125
:101E40000621204698470623D8E7000090F84C204A
:101E5000152A38B5044622D80123934040F6416242
:101E600013421DD113F480150FD19B0217D50B23FC
:101E700080F84C30202383F311882B462A462946CC
:101E8000FFF7D6FD85F3118838BDC3689B695B6891
:101E90002BB9836D03B19847002384F84C3038BDCB
:101EA000002101F0CDF90021204601F0BFF963685F
:101EB0001B6813B10621204698470623EDE7000072
:101EC000024B00221B605B609A607047EC28002088
:101ED000002303748268054B1B6899689142FBD20A
:101EE0005A6803604260106058607047EC28002018
:101EF00008B5202383F31188037C032B05D0042B22
:101F00000DD02BB983F3118808BD436900221A60F4
:101F10004FF0FF334361FFF7DBFF0023F2E790E868
:101F20000C001A6002685360F2E70000002303749B
:101F30008268054B1B6899689142FBD85A68036018
:101F40004260106058607047EC280020054B19690A
:101F50000874186802681A605360186101230374DA
:101F6000FEF7D2B9EC28002030B54B1C87B00546EF
:101F70000A4C10D023690A4A01A800F063F92846E8
:101F8000FFF7E4FF049B13B101A800F097F9236960
:101F9000586907B030BDFFF7D9FFF8E7EC280020FB
:101FA000F11E000838B50C4D41612B6981689A68B3
:101FB0009142044603D8BDE83840FFF789BF184670
:101FC000FFF786FF01232C61014623742046BDE8FC
:101FD0003840FEF799B900BFEC280020044B1A687E
:101FE0001B6990689B68984294BF0020012070474D
:101FF000EC28002010B5084C236820691A6822607C
:102000005460012223611A74FFF790FF0146206992
:10201000BDE81040FEF778B9EC280020FEE700008C
:1020200010B5174CFFF74CFF00F0FEF88022154961
:10203000204600F083F8012344F8180C0374124B77
:10204000124AD96821F4E0610904090C0A431049D5
:10205000DA60CA6842F08072CA600E490A6842F0CB
:1020600001020A601022DA77202283F8222000235E
:1020700083F3118862B60848BDE8104000F080B8CC
:1020800014290020503C000800ED00E00003FA0590
:10209000F0ED00E0001000E0583C00082DE9F84F9A
:1020A0001F4CDFF88090656904F114074FF00008B9
:1020B000D9F82430266AAA689E1B96421DD34FF099
:1020C000200AAA68236AD5F80CB0134423622B684F
:1020D000BB425F60A6EB02066361C5F80C8001D1CC
:1020E00001F0A4FA88F311882869D8478AF3118887
:1020F0006569AB689E42E4D2DAE76269BA420CD005
:10210000916823628E1B9660A86802282CBF18185D
:10211000981CBDE8F84F01F08FBABDE8F88F00BFFA
:10212000EC280020000C0040034B59685A68521AF2
:102130009042FBD8704700BF001000E0826002228E
:1021400002740022427470478368A3F17C0243F852
:102150000C2C026943F83C2C426943F8382C074A9E
:1021600043F81C2CC26843F8102C022203F8082CF8
:10217000002203F8072CA3F1180070472103000880
:1021800010B5202383F31188FFF7DEFF00210446FA
:10219000FFF708FF002383F31188204610BD0000DD
:1021A000024B1B6958610F20FFF7D0BEEC280020BE
:1021B000202383F31188FFF7F3BF000008B5014621
:1021C000202383F311880820FFF7CEFE002383F33A
:1021D000118808BD49B1064B42681B6918605A60F6
:1021E000136043600420FFF7BFBE4FF0FF3070471D
:1021F000EC2800200368984206D01A6802605060FC
:1022000059611846FFF764BE7047000038B50446B0
:102210000D462068844200D138BD036823605C60AD
:102220004561FFF755FEF4E7054B03F114025A61CF
:102230009A614FF0FF32DA6100221A62704700BFE4
:10224000EC280020F8B503611A4BC2605C6A1A4B97
:102250001A46022952F8145F38BF022195420646F9
:102260001F460AD1586198611C6205604560816013
:102270000819BDE8F84001F0CFB9186AAB68241A14
:102280000C1902D3E41A2D6804E09C4202D22044C7
:1022900001F0D2F9AB689C42F4D86B68736035608A
:1022A0001E606E60B460A9684FF0FF33091BA9601F
:1022B000FB61F8BD000C0040EC28002010B41A4C63
:1022C000234653F8141F814210D0416802680A6007
:1022D000026851609A424FF00001C16003D09368D8
:1022E00081680B4493605DF8044B70470A68626133
:1022F00000209A425360C86003D15DF8044B01F09E
:1023000095B99368886803449360084A206A526AC2
:10231000121A9342E7D9991A012998BF931C1844BD
:102320005DF8044B01F088B9EC280020000C004057
:1023300000207047FEE70000704700004FF0FF30BC
:1023400070470000022906D0032906D0012906485B
:1023500018BF0020704705487047032A9ABF0448F9
:1023600000EBC20000207047443D0008F83C000824
:102370000822002070B59AB001AD064608462946ED
:10238000144600F095F82846FEF7F0FCC0B2431C56
:102390005B0086E818002370032363700023023477
:1023A0001946DAB2904204F1020401D81AB070BDA5
:1023B000EA5C04F8022C04F8011C0133F1E7000088
:1023C00008B5202383F311880348FFF751FA00234F
:1023D00083F3118808BD00BFA82A002010B5044669
:1023E000052916D8DFE801F016150316161D20235F
:1023F00083F311880E4A0121FFF7DEFA20460D4AC9
:102400000221FFF7D9FA0C48FFF7F8F9002383F30C
:10241000118810BD202383F311880748FFF7C4F902
:10242000F4E7202383F311880348FFF7DBF9EDE796
:10243000783C00089C3C0008A82A002038B50C4DC8
:102440000C4C0D492A4604F10800FFF793FF05F1F3
:10245000CA0204F110000949FFF78CFF05F5CA72A2
:1024600004F118000649BDE83840FFF783BF00BFFC
:10247000702F002008220020C83C0008D23C000831
:10248000DD3C000870B5044608460D46FEF76EFCBC
:10249000C6B22046013403780BB9184670BD3246E7
:1024A0002946FEF74BFC0028F3D1012070BD000047
:1024B0002DE9F84F05460C46FEF758FC2C49C6B2EC
:1024C0002846FFF7DFFF08B10436F6B2294928464F
:1024D000FFF7D8FF08B11036F6B2632E0DD8DFF83B
:1024E0009090DFF890A0DFF89880DFF898B0224F46
:1024F0002E7846B92670BDE8F88F29462046BDE8FB
:10250000F84F01F02DBB252E2DD107224946284634
:10251000FEF714FC50B93B6823607B6863603B891D
:102520002381BB7AA37207350B34E1E708225146B9
:102530002846FEF703FCB0B9104BA21C13F8011F8C
:1025400009095B4511F8081002F8021C197801F01E
:102550000F0102F1020211F8081002F8031CEDD17C
:1025600018340835C4E7267001350134C0E700BFD0
:10257000643D0008DD3C00086C3D00080F7AFF1F39
:10258000783D00081B7AFF1FBFF34F8F024AD368C4
:10259000DB03FCD4704700BF003C024008B5094B88
:1025A0001B7873B9FFF7F0FF074B1A69002ABFBF0A
:1025B000064A5A6002F188325A601A6822F4806230
:1025C0001A6008BDCE310020003C0240230167455F
:1025D00008B50B4B1B7893B9FFF7D6FF094B1A6967
:1025E00042F000421A611A6842F480521A601A6876
:1025F00022F480521A601A6842F480621A6008BDA0
:10260000CE310020003C0240172870B513D80B4A89
:102610000B4C137863B90B4E4FF0006144F8231054
:1026200056F823500133182B2944F7D10123137096
:1026300054F8200070BD002070BD00BF3032002073
:10264000D03100208C3D0008014B53F8200070472A
:102650008C3D000818207047172810B5044601D992
:10266000002010BDFFF7D0FF064B53F8243018446C
:10267000C21A0BB9012010BD12680132F0D1043B1F
:10268000F6E700BF8C3D0008172810B5044629D88E
:10269000FFF77AFFFFF782FF1349F323CB600C2388
:1026A000B0FBF3F203FB1200D30143EAC003DBB239
:1026B00043F4007343F002030B610B6943F480336E
:1026C0000B61FFF761FF2046FFF79EFF074B53F8B2
:1026D000241000F0DDF8FFF77BFF2046BDE8104036
:1026E000FFF7BABF002010BD003C02408C3D00083F
:1026F0002DE9F84312F00103154640D18218B2F1DA
:10270000026F3CD22C4B1B6813F0010337D02B4CCB
:10271000FFF744FFF323E360FFF736FF40F20127A2
:10272000032D01D9830713D0244C0F46401A40F2E1
:102730000118EB1B0B44012B00EB0706236924D87F
:1027400023F001032361FFF743FF0120BDE8F88375
:10275000236923F44073236123693B43236151F8C8
:10276000046B0660BFF34F8FFFF70EFF03689E42B6
:1027700008D0236923F001032361FFF729FF00201C
:10278000BDE8F883043D0430CAE723F440732361B5
:10279000236943EA08032361B94637F8023B3380D3
:1027A000BFF34F8FFFF7F0FE3688B9F80030B6B2AE
:1027B000B342BED0DDE700BF00380240003C02401B
:1027C000084908B50B7828B153B9FFF7E7FE012394
:1027D0000B7008BD23B1BDE808400870FFF7F8BED4
:1027E00008BD00BFCE31002010B50244064B0439AD
:1027F000D2B2904200D110BD441C00B253F8200068
:1028000041F8040FE0B2F4E750280040104B30B517
:102810001C6F240407D41C6F44F400741C671C6FE5
:1028200044F400441C670B4C236843F4807323601A
:102830000244094B0439D2B2904200D130BD441C4D
:1028400000B251F8045F43F82050E0B2F4E700BF53
:1028500000380240007000405028004007B50122B7
:1028600001A90020FFF7C0FF019803B05DF804FB49
:1028700013B50446FFF7F2FFA04206D002A90122D9
:1028800041F8044D0020FFF7C1FF02B010BD000069
:1028900070470000034B1B689B0042BF024B0122A4
:1028A0001A7070477438024031320020014B18789A
:1028B000704700BF31320020064A536823F00103FD
:1028C0005360EFF30983683383F30988002383F3AC
:1028D0001188704730EF00E010B5202383F3118892
:1028E000104B5B6813F4006318D0F1EE103AEFF36D
:1028F00009844FF0807344F84C3C0B4BDB6844F880
:10290000083CA4F1680383F30988FFF767FB18B15B
:10291000064B44F8503C10BD054BFAE783F3118891
:1029200010BD00BF00ED00E030EF00E03103000813
:102930003403000870470000FEE70000084A094B16
:1029400009498B4204D3094A0021934205D37047B9
:1029500052F8040F43F8040BF3E743F8041BF4E7C1
:10296000743F0008C4320020C4320020C43200206A
:10297000036F30B500229D68C46E11464FF0FF30E2
:1029800004EB421301329542C3F80019C3F8101941
:10299000C3F80809C3F8001BC3F8101BC3F8080BE1
:1029A000EED24FF00113C4F81C3830BD890141F05C
:1029B0002001016103699B06FCD41220FFF7B4BB20
:1029C000204B03EB80022DE9F047D2F80CE0DD6EDE
:1029D000DEF81420461CD2F800C005EB063605EBE5
:1029E0004018516861450BD3D5F83428012303FA08
:1029F00000F022EA0000C5F834081846BDE8F08768
:102A0000BEF81040ACEB0103A34228BF2346D8F820
:102A10001849A4B2B3EB840F10D894681F46A4F1F0
:102A2000040959F804AFC6F800A0042F01D9043FE7
:102A3000F7E71C440B4494605360D2E70020BDE8E4
:102A4000F08700BF3432002010B5054C2046FEF759
:102A50008FFF4FF0A043E366024B236710BD00BF1A
:102A600034320020103E00080378012B70B5054673
:102A700050D12A4BC46E98421BD1294B5A6B42F05D
:102A800080025A635A6D42F080025A655A6D5A6943
:102A900042F080025A615A6922F080025A610E2186
:102AA00043205B69FEF7CEFB1E4BE3601E4BC4F870
:102AB00000380023C4F8003EC0232360EE6E4FF4BC
:102AC0000413A3633369002BFCDA012333610C2068
:102AD000FFF72AFB3369DB07FCD41220FFF724FB46
:102AE0003369002BFCDA0026A6602846FFF740FF7A
:102AF0006B68C4F81068DB68C4F81468C4F81C6814
:102B00004BB90A4BA3614FF0FF336361A36843F0F5
:102B10000103A36070BD064BF4E700BF3432002010
:102B2000003802404014004003002002003C30C046
:102B3000083C30C0F8B5C46E054600212046FFF7BA
:102B400035FF296F00234FF001128F68C4F8343825
:102B50004FF00066C4F81C284FF0FF3004EB43121E
:102B600001339F42C2F80069C2F8006BC2F808093D
:102B7000C2F8080BF2D20B68EA6E6B67636210232F
:102B80001361166916F01006FBD11220FFF7CCFA7C
:102B9000D4F8003823F4FE63C4F80038A36943F482
:102BA000402343F01003A3610923C4F81038C4F88C
:102BB00014380A4BEB604FF0C043C4F8103B084B8D
:102BC000C4F8003BC4F81069C4F800396B6F03F116
:102BD000100243F480136A67A362F8BDEC3D00085D
:102BE00040800010C26E90F86610D2F8003823F4CE
:102BF000FE6343EA0113C2F8003870472DE9F04143
:102C00000EB200EB86080D46D8F80C100F6807F0DE
:102C10000303022B50D0032B50D03D4A3D4F012BD4
:102C200018BF1746C46E4FEA451E04EB0E03002280
:102C3000C3F8102B8A6905F1100C002A40D04A8A8B
:102C400005F158035B013A43E2500123D4F81C28F4
:102C500003FA0CF31343A6444A69C4F81C38002352
:102C6000CEF8103905F13F03002A39D00A8A898B42
:102C70009208012988BF4A43416F04EB8303561829
:102C800041EA0242466729465A602046FFF78EFE17
:102C9000D8F80C301B8A43EA85531F4305F14803DB
:102CA0005B01E7500123D4F81C2803FA05F515430E
:102CB000C4F81C58BDE8F081174FB3E7174FB1E7D0
:102CC00004EB4613D3F8002B22F40042C3F8002B88
:102CD000D4F81C28012303FA0CF322EA0303BAE711
:102CE00004EB83030E4A5A6004EB4616294620463D
:102CF000FFF75CFED6F8003923F40043C6F800392C
:102D0000D4F81C38012202FA05F523EA0505CFE7BD
:102D100000800010008004100080081000800C105B
:102D200000040002026F12684267FFF721BE000034
:102D30005831C36E49015B5813F4004004D013F4BA
:102D4000001F14BF01200220704700004831C36EED
:102D500049015B5813F4004004D013F4001F14BF62
:102D6000012002207047000000EB8101CB68196A46
:102D70000B6813604B6853607047000000EB8103E1
:102D800030B5DD68AA691368D36019B9402B84BFD8
:102D9000402313606B8A1468C26E1C44013CB4FB70
:102DA000F3F46343033323F0030302EB411043EADC
:102DB000C44343F0C043C0F8103B2B6803F0030347
:102DC000012B09B20ED1D2F8083802EB411013F4EE
:102DD000807FD0F8003B14BF43F0805343F0005392
:102DE000C0F8003B02EB4112D2F8003B43F0044331
:102DF000C2F8003B30BD00002DE9F041244DEE6EDD
:102E000006EB40130446D3F8087BC3F8087B380769
:102E10000AD5D6F81438190706D505EB84032146E0
:102E2000DB6828465B689847FA072FD5D6F8143830
:102E3000DB072BD505EB8403D968CCB98B69488AAD
:102E40005E68B6FBF0F200FB12628AB91868DA68B5
:102E500090420DD2121A83E81400202383F31188C4
:102E60000B482146FFF78AFF84F31188BDE8F08103
:102E7000012303FA04F26B8923EA02036B81CB6816
:102E800023B121460248BDE8F0411847BDE8F08172
:102E90003432002000EB810370B5DD68C36E6C69CD
:102EA0002668E6604A0156BB1A444FF40020C2F877
:102EB00010092A6802F00302012A0AB20ED1D3F8DF
:102EC000080803EB421410F4807FD4F8000914BF03
:102ED00040F0805040F00050C4F8000903EB42126B
:102EE000D2F8000940F00440C2F80009D3F83408D1
:102EF000012202FA01F10143C3F8341870BD19B977
:102F0000402E84BF4020206020682E8A841940F023
:102F10000050013C1A44B4FBF6F440EAC440C6E752
:102F2000F8B504461E48C56E05EB4413D3F808698E
:102F3000C3F80869F10717D5D5F81038DA0713D5A3
:102F400000EB8403D9684B691F68DA68974218D28E
:102F5000D21B00271A605F60202383F3118821466B
:102F6000FFF798FF87F31188330617D5D5F8342873
:102F70000123A340134211D02046BDE8F840FFF7DB
:102F80001FBD012303FA04F2038923EA020303812C
:102F90008B68002BE8D021469847E5E7F8BD00BFD5
:102FA00034320020A0482DE9F84FC56E6E69AB6938
:102FB0001E4016F4805F6E61044605D0FEF74AFDA0
:102FC000BDE8F84FFFF788BC002E12DAD5F8003EB6
:102FD00095489B071EBFD5F8003E23F00303C5F8B4
:102FE000003ED5F8043823F00103C5F80438FEF795
:102FF0005DFD370502D58C48FEF74CFDB0040CD5BD
:10300000D5F8083813F0060FEB6823F470530CBFA3
:1030100043F4105343F4A053EB60310704D56368C5
:10302000DB680BB180489847F2026FD4B3020CD52D
:10303000D4F86C80DFF8F0A100274FF00109236F6E
:103040009B68F9B28B4280F09C80F70619D5E16E3F
:103050000A6AC2F30A1702F00F0302F4F012B2F583
:10306000802F00F0B680B2F5402F0AD104EB830325
:1030700001F58051DB68186A00231A469F4240F030
:103080009C803303D5F818481DD5E70302D50020EE
:10309000FFF7B2FEA50302D50120FFF7ADFE6003E6
:1030A00002D50220FFF7A8FE210302D50320FFF777
:1030B000A3FEE20202D50420FFF79EFEA30202D582
:1030C0000520FFF799FE77037FF57AAFE60702D573
:1030D0000020FFF725FFA50702D50120FFF720FFFD
:1030E000600702D50220FFF71BFF210702D503204E
:1030F000FFF716FFE20602D50420FFF711FFA30633
:103100007FF55EAF0520FFF70BFF59E7D4F86C8021
:10311000DFF814A100274FF00109236F9B685FFAC5
:1031200087FB5B4582D308EB4B13D3F8002902F4ED
:103130004022B2F5802F22D1D3F80029002A1EDACE
:10314000D3F8002942F09042C3F80029D3F80029AF
:10315000002AFBDB5946E06EFFF728FC228909FABA
:103160000BF322EA0303238104EB8B03DB689B68E8
:1031700013B15946504698475846FFF721FC01378E
:10318000CBE708EB4112D2F8003B03F44023B3F540
:10319000802F10D1D2F8003B002B0CDA628909FA9B
:1031A00001F322EA0303638104EB8103DB68DB683C
:1031B0000BB150469847013741E79C0708BF0A68A2
:1031C000072B98BF027003F101039CBF120A013064
:1031D00054E7023304EB830201F580515268906991
:1031E0000268D0F808C04068A2EB000E002210462A
:1031F00097420AD104EB830463689B699A683A4456
:103200009A605A6817445F603BE712F0030F08BFEB
:103210000868964588BF8CF8000002F1010284BF5F
:10322000000A0CF1010CE3E734320020C36E03EB1B
:103230004111D1F8003B43F40013C1F8003B704743
:10324000C36E03EB4111D1F8003943F40013C1F808
:1032500000397047C36E03EB4111D1F8003B23F4F2
:103260000013C1F8003B7047C36E03EB4111D1F866
:10327000003923F40013C1F80039704730B5039CBE
:103280000172043304FB0325C361049B0363002123
:10329000059B00604060C16042610261856104621B
:1032A00042628162C162436330BD00000022416A14
:1032B00041610161C2608262C2626FF00101FEF78A
:1032C000A5BF000003694269934203D1C2680AB1F5
:1032D00000207047181D704703691960C2680132E9
:1032E000C260C269134482690361934224BF436A86
:1032F00003610021FEF77EBF38B504460D46E36842
:103300003BB16269131D1268A3621344E36200209B
:1033100038BD237A33B929462046FEF75BFF0028E3
:10332000EDDA38BD6FF00100FBE70000C368C26949
:10333000013BC3604369134482694361934224BFE4
:10334000436A436100238362036B03B118477047EC
:1033500070B52023044683F31188866A3EB9FFF7CF
:10336000CBFF054618B186F31188284670BDA36AC5
:10337000E26A13F8015BA362934202D32046FFF78F
:10338000D5FF002383F31188EFE700002DE9F84F04
:1033900004460E4690469946202787F3118800255B
:1033A000AA46D4F828B0BBF1000F09D149462046FF
:1033B000FFF7A2FF20B18BF311882846BDE8F88FF4
:1033C000A16AE36AA8EB050B5B1A9B4528BF9B46E5
:1033D000BBF1400F1BD9334601F1400251F8040BF9
:1033E00043F8040B9142F9D1A36A40334036A362FB
:1033F0004035A26AE36A9A4202D32046FFF796FF5D
:103400008AF311884545D8D287F31188C9E7304639
:103410005A46FDF789FCA36A5B445E44A3625D449F
:10342000E7E7000010B5029C0172043303FB04219E
:10343000C36100238362C362039B0363049B006038
:103440004060C46042610261816104624262436320
:1034500010BD0000026AC260426A4261026100223D
:103460008262C2626FF00101FEF7D0BE4369026959
:103470009A4203D1C2680AB100207047184650F83A
:10348000043B0B6070470000C368C2690133C3602E
:103490004369134482694361934224BF436A436191
:1034A0000021FEF7A7BE000038B504460D46E368CC
:1034B0003BB123691A1DA262E2691344E362002052
:1034C00038BD237A33B929462046FEF783FE00280B
:1034D000EDDA38BD6FF00100FBE700000369196009
:1034E000C268013AC260C2691344826903619342AF
:1034F00024BF436A036100238362036B03B118474F
:103500007047000070B5202304460E4683F31188EF
:10351000856A35B91146FFF7C7FF10B185F31188E9
:1035200070BDA36A1E70A36AE26A01339342A3626C
:1035300004D3E16920460439FFF7D0FF002080F36F
:10354000118870BD2DE9F84F04460D4691469A4604
:103550004FF0200888F311880026B346A76A4FB9B8
:1035600051462046FFF7A0FF20B187F3118830466F
:10357000BDE8F88FA06AE76AA9EB06033F1A9F42ED
:1035800028BF1F46402F1BD905F1400355F8042BD7
:1035900040F8042B9D42F9D1A36A4033A362403620
:1035A000A26AE36A9A4204D3E16920460439FFF72C
:1035B00095FF8BF311884E45D9D288F31188CDE75A
:1035C00029463A46FDF7B0FBA36A3B443D44A3625B
:1035D0003E44E5E7026943699A4203D1C3681BB9D7
:1035E000184670470023FBE7836A002BF8D0043BA2
:1035F0009B1AF5D01360C368013BC360C3691A44CA
:10360000836902619A4224BF436A03610023836293
:103610000123E5E700F0B2B8034B002258631A61BA
:103620000222DA60704700BF000C0040014B00220C
:10363000DA607047000C0040014B5863704700BFD0
:10364000000C00404B6843608B688360CB68C360AC
:103650000B6943614B6903628B6943620B680360CA
:103660007047000008B5274B27481A6940F2FF71E0
:103670000A431A611A6922F4FF6222F007021A61F2
:103680001A691A6B0A431A631A6D0A431A651F4AAC
:103690001B6D1146FFF7D6FF1D4802F11C01FFF715
:1036A000D1FF1C4802F13801FFF7CCFF1A4802F1A4
:1036B0005401FFF7C7FF194802F17001FFF7C2FF7D
:1036C000174802F18C01FFF7BDFF164802F1A8016F
:1036D000FFF7B8FF144802F1C401FFF7B3FF134826
:1036E00002F1E001FFF7AEFF114802F1FC01FFF724
:1036F000A9FF104802F58C71FFF7A4FFBDE8084050
:1037000000F0A8B800380240000002401C3E00084B
:103710000004024000080240000C02400010024079
:103720000014024000180240001C02400020024029
:10373000002402400028024008B500F0FFF9FEF71F
:103740006FFCFFF7A7F8BDE80840FEF777BE000062
:1037500070470000084B1A69920710B508D500247D
:103760001C61202383F31188FEF798FC84F31188F1
:10377000BDE81040FFF7B0B8000C0040104B1A6CC9
:1037800042F008021A641A6E42F008021A660D4AE4
:103790001B6E936843F0080393600B4B53229A62AD
:1037A0004FF0FF32DA6200229A615A63DA605A609F
:1037B00001225A6108211A603220FDF743BD00BF83
:1037C00000380240002004E0000C00401F4B1A6942
:1037D0006FEA42526FEA52521A611A69C2F30A0240
:1037E0001A614FF0FF301A695A69586100215A690D
:1037F00059615A691A6A62F080521A621A6A02F0B2
:1038000080521A621A6A5A6A58625A6A59625A6A25
:103810001A6C42F080521A641A6E42F080521A6694
:103820001A6E0B4A106840F480701060186F00F434
:103830004070B0F5007F1EBF4FF4803018671967E5
:10384000536823F40073536000F058B90038024005
:1038500000700040324B4FF080521A64314A4FF4EE
:10386000404111601A6842F001021A601A6892071A
:10387000FCD59A6822F003029A60294B19469A688F
:1038800012F00C02FBD1186800F0F90018609A6081
:103890001A6842F480321A600B689B03FCD54B6FA8
:1038A00043F001034B671E4B5A6F9007FCD51E4A2D
:1038B0005A601A6842F080721A601A4A53685904B2
:1038C000FCD5174B1A689201FCD5184A9A6003225E
:1038D000C3F88C20164B1A68164B9A42164B1BD114
:1038E000164A1168164A914216D140F205121A6022
:1038F0000B4B9A6842F002029A609A6802F00C023E
:10390000082AFAD15A6C42F480425A645A6E42F440
:1039100080425A665B6E704740F20572E7E700BF6F
:103920000038024000700040185440070094883866
:10393000002004E011640020003C024000ED00E0A3
:1039400041C20F41084A08B5536911680B4003F0A2
:103950000103536123B1054A13680BB150689847BE
:10396000BDE80840FEF7B8BF003C01409C230020A2
:10397000084A08B5536911680B4003F0020353610C
:1039800023B1054A93680BB1D0689847BDE8084059
:10399000FEF7A2BF003C01409C230020084A08B566
:1039A000536911680B4003F00403536123B1054AC6
:1039B00013690BB150699847BDE80840FEF78CBF0A
:1039C000003C01409C230020084A08B55369116857
:1039D0000B4003F00803536123B1054A93690BB10F
:1039E000D0699847BDE80840FEF776BF003C01402B
:1039F0009C230020084A08B5536911680B4003F066
:103A00001003536123B1054A136A0BB1506A9847FA
:103A1000BDE80840FEF760BF003C01409C23002049
:103A2000174B10B55C691A68144004F478725A6137
:103A3000A30604D5134A936A0BB1D06A984760066F
:103A400004D5104A136B0BB1506B9847210604D56F
:103A50000C4A936B0BB1D06B9847E20504D5094A29
:103A6000136C0BB1506C9847A30504D5054A936CB1
:103A70000BB1D06C9847BDE81040FEF72DBF00BFDA
:103A8000003C01409C2300201A4B10B55C691A6869
:103A9000144004F47C425A61620504D5164A136D41
:103AA0000BB1506D9847230504D5134A936D0BB1A4
:103AB000D06D9847E00404D50F4A136E0BB1506ED9
:103AC0009847A10404D50C4A936E0BB1D06E984769
:103AD000620404D5084A136F0BB1506F9847230452
:103AE00004D5054A936F0BB1D06F9847BDE81040DD
:103AF000FEF7F2BE003C01409C230020062108B5E1
:103B00000846FDF79FFB06210720FDF79BFB0621DA
:103B10000820FDF797FB06210920FDF793FB0621FE
:103B20000A20FDF78FFB06211720FDF78BFB0621EE
:103B30002820BDE80840FDF785BB000008B5FFF769
:103B400045FEFDF72FFAFDF723FDFDF70FFFFDF70B
:103B5000E3FDFFF7FDFDBDE80840FFF75BBD00009A
:103B6000034611F8012B03F8012B002AF9D1704705
:103B7000121012131211000053544D3332463F3FBE
:103B80003F00000000000000783B00083F000000FC
:103B900013040000C03B00083F00000019040000AF
:103BA000CA3B00083F00000021040000D43B00088D
:103BB0003F000000A82A00201C24002084260020AA
:103BC00053544D3332463430780053544D333246DB
:103BD0003432780053544D3332463434365858001A
:103BE000009600000000000000000000000000003F
:103BF00000000000000000005915000845150008ED
:103C0000811500086D150008791500086515000874
:103C1000511500083D1500088D1500080000000032
:103C2000911600087D160008B9160008A5160008B0
:103C3000B11600089D1600088916000875160008C0
:103C4000151700080000000001000000000000003F
:103C50006D61696E00000000703C00083029002092
:103C6000A82A0020010000001D200008000000001C
:103C700069646C65000000000200000000000000A4
:103C8000BD1800082519000840004000402F002002
:103C9000502F002002000000000000000300000080
:103CA000000000006919000800000000100000007A
:103CB000602F002000000000010000000000000054
:103CC00034320020010102004172647550696C6F4A
:103CD000740025424F415244252D424C0025534546
:103CE0005249414C25000000DD230008452300080F
:103CF00029180008C123000843000000003D000807
:103D000009024300020100C032090400000102025E
:103D10000100052400100105240100010424020211
:103D20000524060001070582030800FF09040100BD
:103D3000020A000000070501024000000705810299
:103D400040000000120000004C3D0008120110016C
:103D50000200004009124157000201020301000065
:103D60000403090425424F415244250044726F74F4
:103D7000656B503350726F00303132333435363723
:103D800038394142434445460000000000400000ED
:103D90000040000000400000004000000000010062
:103DA000000002000000020000000200000002000B
:103DB00000000200000002000000020000400000BD
:103DC0000040000000400000004000000000010032
:103DD00000000200000002000000020000000200DB
:103DE00000000200000002000000020000000000CD
:103DF000C11A0008A11D00084D1E00084000400027
:103E0000AC320020AC32002001000000BC320020A7
:103E10008000000040010000050000000000802A32
:103E200000020000AAAAAAAA00000000FFFF0000EA
:103E30000000000000A00A00040040000000000094
:103E4000AAAAAAAA00000000FFFF000000000000CC
:103E5000000000001000004000000000AAAAAAAA6A
:103E600010000040FFFF0000000000000000000004
:103E700080699A0100000000AAAAAAAA405555012B
:103E8000FFFF000000707007777000000000004026
:103E900000000000AAAAAAAA00000040FFFF00003C
:103EA0000000000000000000000000000000000012
:103EB000AAAAAAAA00000000FFFF0000000000005C
:103EC000000000000000000000000000AAAAAAAA4A
:103ED00000000000FFFF00000000000000000000E4
:103EE0000004000000000000AAAA00000004000076
:103EF000FF000000000000000000000000000000C3
:103F000000000000AAAAAA0000000000FF0F0000A5
:103F100000000000000000000000000000000000A1
:103F20000000000000000000000000000000000091
:103F30000000000000000000000000000000000081
:103F40000000000000000000000000000000000071
:103F5000FF0096000000000804000000603D00081B
:103F60000000000000000000000000000000000051
:083F7000000000000000000049
:00000001FF
